:100000006F00C05A1300000013000000130000002E
:100010001300000013000000130000001300000094
:100020001300000013000000130000001300000084
:08003000130000007300100032
:100038000000000000000000280200003802000054
:10004800000000003605000000000000000000006D
:10005800380500003A05000000000000000000001C
:100068003C050000000000003E0500000000000004
:100078004005000042050000440500004605000058
:10008800480500004A0500004C0500004E05000028
:1000980050050000520500005405000056050000F8
:1000A800580500005A0500005C0500005E050000C8
:1000B8006005000062050000640500006605000098
:1000C800680500006A0500006C0500006E05000068
:1000D8007005000072050000740500007605000038
:1000E800780500007A0500007C0500007E05000008
:1000F80080050000820500008405000086050000D8
:10010800880500008A0500008C0500008E050000A7
:100118009005000092050000940500009605000077
:10012800980500009A0500009C0500009E05000047
:10013800A0050000A2050000A4050000A605000017
:10014800A8050000AA05000000000000000000004B
:100158000000000000000000000000000000000097
:100168000000000000000000000000000000000087
:0801780000000000000000007F
:100180003D432A876373C3029377F700BDEFADE564
:10019000937606FF3D8ABA960CC34CC30CC74CC776
:1001A0004107E36BD7FE11E28280B306C3408A06A3
:1001B0009702000096966780A6002307B700A30663
:1001C000B7002306B700A305B7002305B700A304B3
:1001D000B7002304B700A303B7002303B700A302AB
:1001E000B7002302B700A301B7002301B700A300A3
:1001F000B7002300B700828093F5F50F9396850032
:10020000D58D93960501D58D61B7939627009702FA
:10021000000096968682E78086FA9680C1171D8F29
:100220003E96E374C3F8A5B7411122C60008010049
:100230003244410173002030411122C6000801A060
:10024000011106CE22CC00100945EF00B000EF10DE
:10025000E075F16713850720EF10F001B707002064
:1002600083A70707BE858D671385C746EF20C004A7
:10027000EF105015EF10503D232204FE232404FEFE
:10028000232604FE2945EF10C0768D671385C747E6
:10029000EF20C01383C78181850713F7F70F238CE5
:1002A000E18083C79181850713F7F70FA38CE18065
:1002B00083C7A181850713F7F70F238DE18083C7DB
:1002C0008181858B93F7F70F81C70145EF10D02E01
:1002D00003C791818D47B377F70293F7F70F81C773
:1002E0000545EF10702D03C7A1819547B377F7023D
:1002F00093F7F70F81C70945EF10102C9305803E47
:10030000B717004013850780EF10E0379305C0440E
:10031000B717004013850780EF1000399305004B95
:1003200037050040EF10E03193054051370500409C
:10033000EF1040339305805737050040EF10A0348D
:100340009305C05D37050040EF1000369305800C23
:10035000B707004013850740EF10A02E9305C01289
:10036000B707004013850740EF10C02F9305001911
:10037000B707004013850740EF10E0309305401F9A
:10038000B707004013850740EF100032E5BD41116B
:1003900006C622C40008B71702409843B7170240A8
:1003A0001367170098C3B7170240D443B71702402A
:1003B0003707FFF8758FD8C3B71702409443B717B4
:1003C00002403707F7FE7D17758F98C3B7170240B5
:1003D0009443B71702403707FCFF7D17758F98C30A
:1003E000B7170240D443B7170240370781FF7D1784
:1003F000758FD8C3B717024037079F0098C73120C1
:100400000100B240224441018280411106C622C44B
:10041000000831200100B2402244410182800111D4
:1004200022CE0010232604FE232404FEB717024028
:100430009443B71702404167558F98C3B7170240DE
:100440009843B7070200F98F2324F4FE8327C4FEE4
:1004500085072326F4FE832784FE91E70327C4FE45
:100460008567E31DF7FCB71702409843B707020002
:10047000F98F89C785472324F4FE19A0232404FE9D
:10048000032784FE85476312F70A37170240B71720
:1004900002405843D8C337170240B71702405843A9
:1004A000D8C3B7170240D843B717024013670740B5
:1004B000D8C3B7170240D443B71702403707C1FF6C
:1004C0007D17758FD8C3B7170240D443B7170240C2
:1004D00037072900558FD8C3B71702409443B71781
:1004E000024037070001558F98C30100B71702403B
:1004F0009843B7070002F98FF5DBB7170240D843DE
:10050000B7170240719BD8C3B7170240D843B7173B
:10051000024013672700D8C30100B7170240DC432D
:1005200013F7C700A147E31AF7FE01007244056103
:10053000828001A001A001A001A001A001A001A052
:1005400001A001A001A001A001A001A001A001A0A3
:1005500001A001A001A001A001A001A001A001A093
:1005600001A001A001A001A001A001A001A001A083
:1005700001A001A001A001A001A001A001A001A073
:1005800001A001A001A001A001A001A001A001A063
:1005900001A001A001A001A001A001A001A001A053
:1005A00001A001A001A001A001A001A097010020CD
:1005B0009381412C178100201301C1A4173500003D
:1005C000130585F8970500209385C5A313868181BF
:1005D00063FAC5008322050023A05500110591058B
:1005E000E3EAC5FE138581819385C1876377B500F2
:1005F000232005001105E36DB5FEFD42739002BC9A
:100600008D42739042809302800873A0023097025B
:1006100000009382A2A293E2320073905230EFF076
:100620001FD7970200009382E2C1739012347300C7
:100630002030397122DE80002326A4FC2324B4FC60
:10064000232604FE232004FE232404FE232E04FC80
:10065000232204FE232C04FC832784FC9C47BD8BAF
:100660002326F4FE832784FC9C47C18B89CB8327F8
:1006700084FCDC430327C4FED98F2326F4FE8327A2
:1006800084FC9E2393F7F70FE9CF8327C4FC9C4398
:100690002322F4FE232404FE5DA8832784FE05475D
:1006A000B317F700232EF4FC832784FC9E233E8798
:1006B0008327C4FDF98F2320F4FE032704FE83273C
:1006C000C4FD6311F708832784FE8A07232EF4FCF8
:1006D0008327C4FD3D47B317F700232CF4FC832781
:1006E00084FD93C7F7FF032744FEF98F2322F4FE0E
:1006F0008327C4FD0327C4FEB317F700032744FE76
:10070000D98F2322F4FE832784FC98479307800225
:10071000631BF700832784FE05473317F700832701
:10072000C4FCD8CB05A0832784FC9847930780049A
:10073000631AF700832784FE05473317F7008327E2
:10074000C4FC98CB832784FE85072324F4FE03276B
:1007500084FE9D47E3F3E7F48327C4FC032744FEAC
:1007600098C3832784FC9A239307F00F63F0E70E66
:100770008327C4FCDC432322F4FE232404FE6DA85B
:10078000832784FEA1070547B317F700232EF4FC47
:10079000832784FC9E233E878327C4FDF98F232073
:1007A000F4FE032704FE8327C4FD6312F7088327A2
:1007B00084FE8A07232EF4FC8327C4FD3D47B3172C
:1007C000F700232CF4FC832784FD93C7F7FF03274E
:1007D00044FEF98F2322F4FE8327C4FD0327C4FEC1
:1007E000B317F700032744FED98F2322F4FE832793
:1007F00084FC984793078002631BF700832784FEDD
:10080000A10705473317F7008327C4FCD8CB8327FC
:1008100084FC984793078004631BF700832784FEBA
:10082000A10705473317F7008327C4FC98CB83271C
:1008300084FE85072324F4FE032784FE9D47E3F10D
:10084000E7F48327C4FC032744FED8C30100725495
:1008500021618280011122CE00102326A4FEAE87E2
:100860002322C4FE2315F4FE832744FE99C70357B1
:10087000A4FE8327C4FE98CB31A00357A4FE832790
:10088000C4FED8CB0100724405618280797122D602
:100890000018232EA4FC232CB4FC232404FE2322C2
:1008A00004FE232604FE232004FE8327C4FD63D810
:1008B0000700B7070140DC4F2326F4FE31A0B7073D
:1008C0000140DC432326F4FE8327C4FDC183BD8B96
:1008D0002320F4FE0327C4FDC167FD17F98F2324ED
:1008E000F4FE8327C4FD63D407080327C4FDB707BC
:1008F00030007D8FB70730006314F702832704FEB2
:10090000C1070D47B317F7002322F4FE832744FEE7
:1009100093C7F7FF0327C4FEF98F2326F4FEC5A86B
:100920000327C4FDB7071000F98F95C3832704FE82
:100930000D47B317F7002322F4FE832744FE93C725
:10094000F7FF0327C4FEF98F2326F4FEC9A08327EF
:10095000C4FDD5839207032784FEB317F70093C71E
:10096000F7FF0327C4FEF98F2326F4FE4DA00327CB
:10097000C4FDB70730007D8FB70730006315F7025D
:100980000327C4FEB70700F1FD17F98F2326F4FEF5
:10099000B7070140D443B7070140370700F17D177F
:1009A000758FD8C3ADA00327C4FDB7071000F98F1A
:1009B0008DCB832704FE0D47B317F7002322F4FEE7
:1009C000832744FE93C7F7FF0327C4FEF98F23262E
:1009D000F4FE0327C4FEB707000FD98F2326F4FEC9
:1009E0003DA08327C4FDD5839207032784FEB31758
:1009F000F70093C7F7FF0327C4FEF98F2326F4FE01
:100A00000327C4FEB707000FD98F2326F4FE8327E0
:100A100084FD91CF8327C4FDD5839207032784FEED
:100A2000B317F7000327C4FED98F2326F4FE8327CC
:100A3000C4FD63D80700B70701400327C4FED8CF21
:100A400031A0B70701400327C4FED8C301003254C8
:100A500045618280011122CE00102326A4FE0327C7
:100A6000C4FE23AEE1800100724405618280797189
:100A700022D60018232EA4FC232404FE232604FEE1
:100A8000232204FE232004FEB7170240DC43B18B6F
:100A90002324F4FE032784FE91476303F702032710
:100AA00084FEA1476306F702832784FE639607103E
:100AB0008327C4FD37177A001307072098C329A29C
:100AC0008327C4FD3757E8011307078098C3EDA8B3
:100AD000B7170240D843B7073C00F98F2326F4FE2E
:100AE000B7170240D843C167F98F2322F4FE83274A
:100AF000C4FEC98389072326F4FE0327C4FEC54725
:100B00006315F700C9472326F4FE832744FEA1E3BB
:100B1000B7470240938707809C43C18B89CF032747
:100B2000C4FEB7177A00938707203307F70283279D
:100B3000C4FD98C351A80327C4FEB7173D0093878F
:100B400007903307F7028327C4FD98C3B5A8B717EA
:100B50000240D843B707C0007D8FB707C000631EAF
:100B6000F7000327C4FEB727F40093870740330735
:100B7000F7028327C4FD98C381A8B7170240D84362
:100B8000B7070200F98F89CF0327C4FEB7173D00CE
:100B9000938707903307F7028327C4FD98C32DA0DE
:100BA0000327C4FEB7177A00938707203307F7029D
:100BB0008327C4FD98C309A88327C4FD37177A008B
:100BC0001307072098C30100B7170240DC4393F7CF
:100BD000070F2324F4FE832784FE91832324F4FE4D
:100BE000B707002013870700832784FEBA979C234A
:100BF00093F7F70F2320F4FE8327C4FD9843832740
:100C000004FE3357F7008327C4FDD8C3B71702404B
:100C1000DC4393F707702324F4FE832784FEA1832B
:100C20002324F4FEB707002013870700832784FEE0
:100C3000BA979C2393F7F70F2320F4FE8327C4FD74
:100C4000D843832704FE3357F7008327C4FD98C792
:100C5000B7170240D843916793870780F98F232401
:100C6000F4FE832784FEAD832324F4FEB70700201F
:100C700013870700832784FEBA979C2393F7F70F07
:100C80002320F4FE8327C4FDD843832704FE335773
:100C9000F7008327C4FDD8C7B7170240D843B16710
:100CA000F98F2324F4FE832784FEB9832324F4FEE2
:100CB000B707002013874707832784FEBA979C2332
:100CC00093F7F70F2320F4FE8327C4FDD84783272B
:100CD00004FE3357F7028327C4FD98CB010032543A
:100CE00045618280011122CE00102326A4FE232418
:100CF000B4FE832784FE99CBB7170240944FB717F1
:100D000002400327C4FE558F98CF21A8B717024091
:100D1000944F8327C4FE13C7F7FFB7170240758FA0
:100D200098CF0100724405618280011122CE00102B
:100D30002326A4FE2324B4FE832784FE99CBB71771
:100D40000240D44FB71702400327C4FE558FD8CFB7
:100D500021A8B7170240D44F8327C4FE13C7F7FF5B
:100D6000B7170240758FD8CF0100724405618280A9
:100D7000797122D60018232EA4FC232CB4FC23174F
:100D800004FE8327C4FD9E232317F4FE0327C4FD1E
:100D9000B7370140938707C06300F7040327C4FDFA
:100DA000B7070040630AF7020327C4FDB7070040F6
:100DB000938707406302F7020327C4FDB71700407B
:100DC00093870780630AF7000327C4FDB717004025
:100DD000938707C06310F7028357E4FE93F7F7F891
:100DE0002317F4FE832784FDBA238357E4FED98FAB
:100DF0002317F4FE8357E4FE93F7F7CF2317F4FE8F
:100E0000832784FDFA238357E4FED98F2317F4FE4A
:100E10008327C4FD0357E4FE9AA3832784FDDA23C6
:100E20008327C4FDDAB7832784FD9A238327C4FD73
:100E30009AB70327C4FDB7370140938707C0631BE8
:100E4000F700832784FD9C2713970701418383279D
:100E5000C4FD9ABB8327C4FD0547DAAB01003254B9
:100E600045618280797122D60018232EA4FC232CA0
:100E7000B4FC231504FE231704FE231604FE832767
:100E8000C4FD9E33C207C183F99B139707014183B9
:100E90008327C4FD9AB38327C4FD9E332317F4FE32
:100EA0008327C4FDDE232316F4FE8327C4FD9E2F73
:100EB0002315F4FE8357A4FE93F7F7F82315F4FEE9
:100EC0008357A4FEF19B2315F4FE832784FD9A2308
:100ED0008357A4FED98F2315F4FE8357E4FEF59BB8
:100EE0002317F4FE832784FD9A278357E4FED98FC6
:100EF0002317F4FE832784FDBA238357E4FED98F9A
:100F00002317F4FE0327C4FDB7370140938707C0BA
:100F10006318F7068357E4FEDD9B2317F4FE83274F
:100F200084FDBA278357E4FED98F2317F4FE835735
:100F3000E4FEED9B2317F4FE832784FDDA23835719
:100F4000E4FED98F2317F4FE8357C4FE93F7F7EF1F
:100F50002316F4FE8357C4FE93F7F7DF2316F4FE3F
:100F6000832784FDDA278357C4FED98F2316F4FE26
:100F7000832784FDFA278357C4FED98F2316F4FEF6
:100F80008327C4FD0357C4FEDAA38327C4FD035798
:100F9000A4FE9AAF832784FDFA238327C4FDDABB1E
:100FA0008327C4FD0357E4FE9AB301003254456120
:100FB0008280797122D60018232EA4FC232CB4FC45
:100FC000231504FE231704FE231604FE8327C4FD05
:100FD0009E33C207C183BD9B1397070141838327BB
:100FE000C4FD9AB38327C4FD9E332317F4FE8327E1
:100FF000C4FDDE232316F4FE8327C4FD9E2F231594
:10100000F4FE0357A4FEE577FD17F98F2315F4FED0
:101010008357A4FE93F7F7CF2315F4FE832784FDAF
:101020009E23A2071397070141838357A4FED98FFC
:101030002315F4FE8357E4FE93F7F7FD2317F4FE20
:10104000832784FD9E2792071397070141838357C7
:10105000E4FED98F2317F4FE832784FDBE23920775
:101060001397070141838357E4FED98F2317F4FEBA
:101070000327C4FDB7370140938707C0631CF708F7
:101080008357E4FE93F7F7F72317F4FE832784FDD5
:10109000BE2792071397070141838357E4FED98F38
:1010A0002317F4FE8357E4FE93F7F7FB2317F4FEB0
:1010B000832784FDDE23920713970701418383571B
:1010C000E4FED98F2317F4FE8357C4FE93F7F7BFCE
:1010D0002316F4FE0357C4FEFD779387F77FF98F3D
:1010E0002316F4FE832784FDDE278A071397070162
:1010F00041838357C4FED98F2316F4FE832784FDD2
:10110000FE278A071397070141838357C4FED98FAF
:101110002316F4FE8327C4FD0357C4FEDAA38327F6
:10112000C4FD0357A4FE9AAF832784FDFA238327C7
:10113000C4FD9ABF8327C4FD0357E4FE9AB30100A0
:10114000325445618280797122D60018232EA4FC86
:10115000232CB4FC231504FE231704FE231604FEDF
:101160008327C4FD9E33C207C18393F7F7EF13971C
:10117000070141838327C4FD9AB38327C4FD9E33AF
:101180002317F4FE8327C4FDDE232316F4FE8327F2
:10119000C4FDDE2F2315F4FE8357A4FE93F7F7F862
:1011A0002315F4FE8357A4FEF19B2315F4FE832739
:1011B00084FD9A238357A4FED98F2315F4FE835709
:1011C000E4FE93F7F7DF2317F4FE832784FD9E27C1
:1011D000A2071397070141838357E4FED98F231792
:1011E000F4FE832784FDBE23A207139707014183E2
:1011F0008357E4FED98F2317F4FE0327C4FDB737C6
:101200000140938707C0631EF7080357E4FEFD778C
:101210009387F77FF98F2317F4FE832784FDBE277A
:10122000A2071397070141838357E4FED98F231741
:10123000F4FE8357E4FE93F7F7BF2317F4FE8327EA
:1012400084FDDE23A2071397070141838357E4FE41
:10125000D98F2317F4FE0357C4FEFD77FD17F98FCE
:101260002316F4FE0357C4FEF977FD17F98F2316F2
:10127000F4FE832784FDDE2792071397070141833D
:101280008357C4FED98F2316F4FE832784FDFE27DF
:1012900092071397070141838357C4FED98F231602
:1012A000F4FE8327C4FD0357C4FEDAA38327C4FDDD
:1012B0000357A4FEDAAF832784FDFA238327C4FDF6
:1012C000DABF8327C4FD0357E4FE9AB3010032540A
:1012D00045618280797122D60018232EA4FC232C2C
:1012E000B4FC231604FE231504FE231704FE8327F3
:1012F000C4FD9E33139707014183FD77FD17F98FD6
:101300001397070141838327C4FD9AB38327C4FD44
:101310009E332315F4FE8327C4FDDE232317F4FE3A
:101320008327C4FDDE2F2316F4FE0357C4FEE577A2
:10133000FD17F98F2316F4FE8357C4FE93F7F7CFFA
:101340002316F4FE832784FD9E23A207139707012B
:1013500041838357C4FED98F2316F4FE0357A4FE9E
:10136000F977FD17F98F2315F4FE832784FD9E2757
:10137000B2071397070141838357A4FED98F231522
:10138000F4FE832784FDBE23B20713970701418330
:101390008357A4FED98F2315F4FE0327C4FDB73766
:1013A0000140938707C06315F7020357E4FEF17706
:1013B000FD17F98F2317F4FE832784FDDE279A0794
:1013C0001397070141838357E4FED98F2317F4FE57
:1013D0008327C4FD0357E4FEDAA38327C4FD035724
:1013E000C4FEDAAF832784FDFA238327C4FD23904C
:1013F000E7048327C4FD0357A4FE9AB301003254C7
:1014000045618280011122CE00102326A4FE2324F0
:10141000B4FE832784FE99CF8327C4FE9E23C20790
:10142000C18393E717001397070141838327C4FE05
:101430009AA329A88327C4FE9E23C207C183F99BD0
:101440001397070141838327C4FE9AA301007244C6
:1014500005618280011122CE00102326A4FE2324E0
:10146000B4FE832784FE95C38327C4FE83D7470435
:10147000139707014183E177D98F139707014183C0
:101480008327C4FE2392E70415A08327C4FE83D7D5
:101490004704139707014183A167FD17F98F13973D
:1014A000070141838327C4FE2392E70401007244AD
:1014B00005618280011122CE00102326A4FE232480
:1014C000B4FE832784FE99CF8327C4FE9E23C207E0
:1014D000C18393E707081397070141838327C4FE5D
:1014E0009AA331A88327C4FE9E23C207C18393F722
:1014F000F7F71397070141838327C4FE9AA30100DE
:10150000724405618280797122D60018232EA4FCD2
:10151000AE87231DF4FC231704FE8327C4FD9E2FF2
:101520002317F4FE8357E4FEDD9B2317F4FE0357D5
:10153000E4FE8357A4FDD98F2317F4FE8327C4FD4F
:101540000357E4FE9AAF01003254456182807971FD
:1015500022D60018232EA4FCAE87231DF4FC2317EB
:1015600004FE8327C4FD9E2F2317F4FE0357E4FED9
:10157000FD779387F77FF98F2317F4FE8357A4FD38
:10158000A2071397070141838357E4FED98F2317DE
:10159000F4FE8327C4FD0357E4FE9AAF01003254E2
:1015A00045618280797122D60018232EA4FCAE8773
:1015B000231DF4FC231704FE8327C4FDDE2F23170D
:1015C000F4FE8357E4FEDD9B2317F4FE0357E4FE8D
:1015D0008357A4FDD98F2317F4FE8327C4FD035737
:1015E000E4FEDAAF0100325445618280797122D67F
:1015F0000018232EA4FCAE87231DF4FC231704FE41
:101600008327C4FDDE2F2317F4FE0357E4FEFD7786
:101610009387F77FF98F2317F4FE8357A4FDA20762
:101620001397070141838357E4FED98F2317F4FEF4
:101630008327C4FD0357E4FEDAAF0100325445614D
:101640008280011122CE00102326A4FEAE8723152E
:10165000F4FE8327C4FE0357A4FEDABB01007244E4
:1016600005618280011122CE00102326A4FEAE87E0
:101670002315F4FE8327C4FE0357A4FE9ABF01007E
:10168000724405618280011122CE00102326A4FE3F
:10169000AE872315F4FE8327C4FE0357A4FEDABFEA
:1016A0000100724405618280011122CE00102326C0
:1016B000A4FEAE872315F4FE8327C4FE0357A4FEC1
:1016C0002390E70401007244056182805D7186C643
:1016D000A2C48008232EA4FA232CB4FA232604FEE5
:1016E000232404FE232204FE232004FE232E04FCD4
:1016F0008327C4FB232EF4FC8327C4FB9E2BC20745
:10170000C1832326F4FE0327C4FEB567FD17F98FB6
:101710002326F4FE832784FBFE233E878327C4FE13
:10172000D98F2326F4FE8327C4FE13970701418334
:101730008327C4FB9AAB8327C4FBDE27C207C18380
:101740002326F4FE0327C4FEBD679387379FF98FD6
:101750002326F4FE832784FBDA23832784FB9E273A
:10176000D98F139707014183832784FBBE27D98F25
:10177000C207C1833E878327C4FED98F2326F4FE88
:101780008327C4FE1397070141838327C4FBDAA78D
:101790008327C4FBDE2BC207C1832326F4FE032765
:1017A000C4FEC1679387F7CFF98F2326F4FE832702
:1017B00084FBDE273E878327C4FED98F2326F4FED1
:1017C0008327C4FE1397070141838327C4FBDAAB49
:1017D000930784FC3E85EFF08FA90327C4FDB7472C
:1017E0000140938707806317F700832744FD232474
:1017F000F4FE29A0832704FD2324F4FE8327C4FBE1
:10180000DE27C207C183C207C18763D2070203274D
:1018100084FEBA878607BA978E073E97832784FB94
:101820009C438607B357F7022322F4FE05A0032743
:1018300084FEBA878607BA978E073E97832784FB74
:101840009C438A07B357F7022322F4FE032744FE82
:1018500093074006B357F70292072326F4FE832727
:10186000C4FE13D7470093074006B307F7020327C8
:1018700044FEB307F7402320F4FE8327C4FBDE2792
:10188000C207C183C207C18763D20702832704FE50
:101890008E071387270393074006B357F7029D8BE4
:1018A0000327C4FED98F2326F4FE05A0832704FE58
:1018B00092071387270393074006B357F702BD8BA0
:1018C0000327C4FED98F2326F4FE8327C4FE139773
:1018D000070141838327C4FB9AA70100B640264431
:1018E00061618280011122CE00102326A4FE2324F0
:1018F000B4FE832784FE85C38327C4FEDE271397A7
:10190000070141838967D98F139707014183832793
:10191000C4FEDAA705A08327C4FEDE2713970701BC
:101920004183F977FD17F98F1397070141838327C7
:10193000C4FEDAA70100724405618280011122CE43
:1019400000102326A4FEAE872315F4FE8357A4FEC1
:1019500093F7F71F1397070141838327C4FEDAA388
:101960000100724405618280797122D60018232E0D
:10197000A4FCAE87231DF4FC232604FE8327C4FDAC
:101980009E231397070141838357A4FDF98FC20754
:10199000C18389C785472326F4FE19A0232604FEA8
:1019A0008327C4FE3E85325445618280411122C6A0
:1019B0000008B707002003A70707B7177A00938727
:1019C0000720B357F70213F7F70F2380E18283C78D
:1019D00001821397070141839307803EB307F70203
:1019E0001397070141832391E182010032444101B1
:1019F0008280797122D60018232EA4FC37F700E0EC
:101A0000544337F700E0F99A54C303D72182BA86CA
:101A10000327C4FD3307D7022326E4FE37F700E08F
:101A20008326C4FEB68701481CCB232A0701B7F7DB
:101A300000E09843B7F700E01367070198C3B7F7D2
:101A400000E09843B7F700E01367170298C301005E
:101A5000B7F700E0DC4313F717008547E31AF7FEFA
:101A6000B7F700E09843B7F700E0799B98C301000F
:101A7000325445618280397106DE22DC80002326E3
:101A8000A4FC8545916713854700EFF0AFA5930748
:101A900000202312F4FE8D472324F4FEE147232681
:101AA000F4FE930744FEBE85B717014013850780F7
:101AB000EFE03FB88327C4FC232AF4FC231C04FC7A
:101AC000231D04FC231E04FC231004FEA147231F36
:101AD000F4FC930744FDBE85B7470140138507809A
:101AE000F5368545B747014013850780E53B010082
:101AF000F250625421618280797106D622D4001896
:101B0000232EA4FC232CB4FC232AC4FC232604FE8D
:101B100081A0010093050004B747014013850780A9
:101B2000A135AA87E5DB832784FD13871700232CC3
:101B3000E4FC83870700C207C183BE85B747014025
:101B400013850780E53B8327C4FE85072326F4FE23
:101B50000327C4FE832744FDE34DF7FA832744FDA2
:101B60003E85B250225445618280011122CE001080
:101B70002326A4FE03A781808327C4FE3E97938774
:101B8000C187636DF70003A781808327C4FE3E975A
:101B9000B78700209387078063F4E700FD5739A8D3
:101BA00003A781808327C4FE3E9723A4E18003A777
:101BB00081808327C4FEB307F040BA973E85724404
:101BC00005618280411106C622C4000801479306C0
:101BD0000008B7170140138607808D679385474932
:101BE000138501831D280147C146371601408D67C3
:101BF00093858749138581840D2001479306000250
:101C0000371601408D679385074A13850186312079
:101C10000100B240224441018280397106DE22DC9B
:101C200080002326A4FC2324B4FC2322C4FCB68712
:101C30002311F4FCBA87A300F4FC232E04FC232018
:101C400004FE232204FE032744FCB71701409387B8
:101C500007806316F70091472326F4FE85A003272B
:101C600044FCB7170140938707C06316F700A147EC
:101C70002326F4FEA1A0032744FCB71701406316F6
:101C8000F700C1472326F4FE15A8032744FCB71725
:101C90000140938707406317F7009307000223264C
:101CA000F4FE29A8032744FCB72701409387078047
:101CB0006316F700930700042326F4FE85450325E9
:101CC000C4FEEFF02F82835724FC231EF4FCC1478F
:101CD0002322F4FE89472320F4FE9307C4FDBE852A
:101CE000032544FCEFE0FF948327C4FC23AA0700EC
:101CF0008327C4FC032784FC98C38327C4FC0357B1
:101D000024FCDAA78327C4FC032744FC98C7832755
:101D1000C4FC238707008327C4FC1307803E98CBAD
:101D2000834714FC8DC38327C4FC98478327C4FCD6
:101D3000DE270146BE853A85EFE0DFB18327C4FC8C
:101D40000547F8A705A08327C4FC98478327C4FC50
:101D5000DE270546BE853A85EFE0DFAF8327C4FC6A
:101D60002387070083A741829DCF83A74182232435
:101D7000F4FE31A0832784FEDC4B2324F4FE83276A
:101D800084FEDC4BE5FB832784FE0327C4FCD8CB11
:101D9000832784FEDE23850713970701418383276A
:101DA000C4FCDAA329A00327C4FC23A2E18201001A
:101DB000F250625421618280797106D622D40018D3
:101DC000AA87231FF4FC83A74182B5CB83A7418256
:101DD0002326F4FE8DA08327C4FEDE230357E4FDF3
:101DE0006316F7048327C4FEFC278DE38327C4FE14
:101DF00098478327C4FEDE270146BE853A85EFE07B
:101E00007FA58327C4FE0547F8A715A88327C4FE2E
:101E100098478327C4FEDE270546BE853A85EFE056
:101E20007FA38327C4FE2387070011A88327C4FE4E
:101E3000DC4B2326F4FE8327C4FED1FF09A001005A
:101E4000B250225445618280411106C622C4000866
:101E50000128BD2219260100B2402244410182809E
:101E6000397106DE22DC8000232204FE232404FED6
:101E7000232604FE232A04FC232C04FC232E04FC2A
:101E8000232004FE232404FC232604FC231804FC42
:101E900085451145EFE01FE585450545EFE0FFE885
:101EA000BD472312F4FEE1472326F4FE8D47232489
:101EB000F4FE930744FEBE85B717014013850780E3
:101EC000EFE02FF7B707002003A70707B7470F007A
:101ED00093870724B357F702C207C183FD17C207D0
:101EE000C1832314F4FC95679387F7E12316F4FC70
:101EF000231704FC231504FC930784FCBE853705D7
:101F00000040EFE0FFE693070006231AF4FC854744
:101F1000231BF4FC231E04FC9307803E231DF4FCCA
:101F2000930744FDBE8537050040EFE0BFF39307FC
:101F3000803E231DF4FC930744FDBE853705004019
:101F4000EFF02F879307803E231DF4FC930744FD99
:101F5000BE8537050040EFF00F9F9307803E231D9D
:101F6000F4FC930744FDBE8537050040EFF08FB6C3
:101F7000A14537050040EFF00FD9A14537050040D6
:101F8000EFF0EFDCA14537050040EFF0AFE1A145F0
:101F900037050040EFF08FE5854537050040EFF04D
:101FA0006FD1854537050040EFF0CFCA854537052D
:101FB0000040EFF02FC50100F25062542161828091
:101FC000397106DE22DC8000232204FE232404FE75
:101FD000232604FE232A04FC232C04FC232E04FCC9
:101FE000232004FE232404FC232604FC231804FCE1
:101FF00085454545EFE01FCF85450945EFE0FFD218
:102000008545B7171A00138507C0EFE03F8893078F
:10201000003C2312F4FEE1472326F4FE8D472324DF
:10202000F4FE930744FEBE8537150140EFE06FE0F4
:10203000B707002003A70707B7470F0093870724B8
:10204000B357F702C207C183FD17C207C183231428
:10205000F4FC9307703E2316F4FC231704FC2315AD
:1020600004FC930784FCBE85B70700401385074036
:10207000EFE01FD093070006231AF4FC8547231BCB
:10208000F4FC231E04FC93074006231DF4FC930775
:1020900044FDBE85B707004013850740EFE09FDC95
:1020A00093074006231DF4FC930744FDBE85B70744
:1020B000004013850740EFE0DFEF93074006231D44
:1020C000F4FC930744FDBE85B70700401385074025
:1020D000EFF06F8793074006231DF4FC930744FD40
:1020E000BE85B707004013850740EFF0AF9EA145BE
:1020F000B707004013850740EFF0EFC0A145B707D1
:10210000004013850740EFF08FC4A145B70700409A
:1021100013850740EFF00FC9A145B70700401385AD
:102120000740EFF0AFCC8545B70700401385074067
:10213000EFF04FB88545B707004013850740EFF033
:102140006FB18545B707004013850740EFF08FABAF
:102150000100F250625421618280397106DE22DC76
:102160008000232204FE232404FE232604FE232AC7
:1021700004FC232C04FC232E04FC232004FE232433
:1021800004FC232604FC231804FC85452145EFE0CC
:102190007FB585451145EFE05FB993070030231205
:1021A000F4FEE1472326F4FE8D472324F4FE930733
:1021B00044FEBE85B7170140138507C0EFE06FC727
:1021C000B707002003A70707B7470F009387072427
:1021D000B357F702C207C183FD17C207C183231497
:1021E000F4FC95679387F7E12316F4FC231704FCAE
:1021F000231504FC930784FCBE85B71700401385A4
:102200000780EFE0FFB693070006231AF4FC85472A
:10221000231BF4FC231E04FC9307803E231DF4FCC7
:10222000930744FDBE85B717004013850780EFE094
:102230009FF19307803E231DF4FC930744FDBE8568
:10224000B717004013850780EFF0CF88A145B71777
:10225000004013850780EFF00FABA145B717004092
:1022600013850780EFF0AFAEA145B7170040138587
:102270000780EFF02FB3A145B71700401385078003
:10228000EFF0CFB68545B717004013850780EFF014
:102290006FA28545B717004013850780EFF08F9B2D
:1022A0008545B717004013850780EFF0AF95010013
:1022B000F25062542161828039713EDA2ED232D4DA
:1022C00036D63AD842DC46DE9387C18022CC8043A2
:1022D00026CA06CEAA8409C41C4C99E32285ED299E
:1022E0000C4454102686228536C6EF007012F24048
:1022F0006244D24421618280011126CA4AC806CEB6
:1023000022CC4EC652C4AA842E8901C51C4D91E32D
:10231000E1219C4C804499E326857D299717000094
:102320009387C71A631BF402C0405E24A18BB1C718
:102330001C48A1C7FD59294A1C4483450900FD17C3
:10234000B1E91CC463DD07062286A9452685612004
:10235000FD576308F502294535A0971700009387BC
:10236000E7186314F4008044C9B7971700009387F7
:10237000E713E31CF4FAC0444DBFA2852685112A59
:1023800055D97D55F2406244D2444249B249224A6D
:10239000056182801CC4050963D70700184C63CA15
:1023A000E700638845011C401387170018C08CA301
:1023B00061B7228626850520E31035F9D9B71C4080
:1023C0001387170018C0294798A371B79387C18056
:1023D000AA85884315B7011122CC26CA4AC806CE61
:1023E0004EC6AA842E89328401C51C4D91E3ED2688
:1023F000971700009387870D6317F406C0401C4CA5
:102400001CC45E24A18BC1C31C48B5CF1C48084026
:102410009379F90F1379F90F1D8D5C486346F50028
:10242000A2852685692C25E51C440505FD171CC4DD
:102430001C401387170018C0238037015C4863884D
:10244000A7005E24858B81CBA9476316F900A2857E
:102450002685B5240DEDF24062444A85D2444249B6
:10246000B24905618280971700009387270863149B
:10247000F400804469B79717000093872703E3109F
:10248000F4F8C044ADBFA2852685212041D17D59F5
:10249000D9B741119387C18026C2844322C44AC060
:1024A00006C62A892E8489C49C4C99E326852D264C
:1024B0009717000093878701631BF402C04003173E
:1024C000C40093170701C18393F68700ADEA93F622
:1024D000070195EEA5472320F900136707045AA4C6
:1024E0007D55B240224492440249410182809717AF
:1024F00000009387A7FF6314F4008044C9B79717BF
:1025000000009387A7FAE31CF4FAC0444DBF918BF7
:102510009DC34C5889C9930744046384F5004A85D8
:102520003123232A04025E242322040093F7B7FDFB
:102530005EA41C481CC05E2493E787005EA41C4870
:1025400099EB5E241307002093F707286385E700C3
:10255000A2854A85A1215E2413F717001DC35C489C
:1025600023240400B307F0401CCC1C480145B5FBF4
:102570008317C40013F707082DD793E707045EA459
:1025800085B7898B014791E3584818C4F9BFDE2508
:10259000011122CC26CA06CE4AC84EC613F78700C0
:1025A000AA842E8479EBD841634DE000B841634A98
:1025B000E0000145F2406244D2444249B24905611B
:1025C000828058547DD703A904009396370123A035
:1025D000040063DB060670485E24918B99C75C405B
:1025E0001D8E5C5899C33C401D8E5C540C50814636
:1025F00026858297FD575A24631DF5009440F547C0
:1026000063E8D706B70740208507B3D7D700858B87
:10261000A5C31C48232204001CC09317370163D8AC
:102620000700FD576314F5009C4091E368C84C58BF
:1026300023A02401BDDD930744046384F5002685AF
:10264000F526232A0402B5B70C5001468546268597
:102650000297FD572A86E311F5F89C40B5DF7547D0
:102660006385E70059476393E70423A0240191B7EA
:10267000136707045AA47D5535BF83A90501E38A72
:1026800009F203A905008D8B23A0350133093941D7
:10269000014791E3D84918C4E35D20F11C540C5064
:1026A000CA864E86268582976347A0005E2493E7FC
:1026B00007045EA4C9B7AA993309A940F1BF9C4990
:1026C000B9CF011122CC06CE2A8411C51C4D81E759
:1026D0002EC61922B24597170000938727DF639B08
:1026E000F5004C408397C50095C722856244F240AF
:1026F000056171BD97170000938747DF6394F5006C
:102700000C44CDB797170000938747DAE39CF5FC9C
:102710004C44C9BFF24062440145056182800145D5
:102720008280411122C406C62A844EA572A52320A8
:102730000500232205002324050023220506232863
:102740000500232A0500232C050021468145130599
:10275000C505EFD0FFA297170000938747B15CD063
:1027600097170000938767B31CD4971700009387CF
:1027700047B75CD4971700009387A7B900D01CD83F
:10278000B24022444101828097050000938565F3A1
:10279000A9A2411126C2130680069384F5FFB384D3
:1027A000C4024AC02E8922C406C6938544071D264A
:1027B0002A8401CD2320050023222501310508C4E8
:1027C000138684068145EFD0BF9B2285B240224408
:1027D00092440249410182801C4DADE3411106C67D
:1027E00022C497070000938767FA1CD5938701815D
:1027F0009C4323240504232605042328050463148D
:10280000F50085471CCD2A841D2848C0228505284F
:1028100008C422852D2048C44840014691451137FF
:1028200008440546A545F53D48440946C945D53DFA
:1028300085471CCCB24022444101828082804111F4
:102840009387018126C284434AC006C69C4C22C499
:102850002A8999E326854937938484048044DC409F
:10286000FD1763D607009C40B9CF8440C5BF03174E
:10287000C40039E7C177850723220406232004001A
:1028800023220400232404005CC423280400232AF8
:102890000400232C0400214681451305C405EFD014
:1028A0003F8E232A0402232C04022324040423261B
:1028B00004042285B24022449244024941018280AC
:1028C0001304840671BF91454A85E13588C051FDE6
:1028D000B1472320F9000144E9BF797122D44AD0DD
:1028E00052CC56CA5AC85EC606D626D24ECE2A8AC0
:1028F000AE8A130485040149054BFD5B09ECB25017
:1029000022544A8592540259F249624AD24A424BB1
:10291000B24B45618280044483294400FD1963D48D
:1029200009000040E1BFDE24637BFB008397E400E5
:1029300063877701A6855285829A3369A9009384BB
:102940008406E9BF1971A6DAAE848395E500A2DC9E
:1029500086DE328463DB0500DE2423A0060093F7C5
:10296000070885E7930700401DA0300836C6EF0032
:10297000D01FB246E34205FE7247BD67F98F7977F3
:10298000BA9793B717009CC2F1BF930700041CC00D
:10299000F6506654D654014509618280DE25011146
:1029A00022CC06CE26CA4AC8898B2E8489CF9307AB
:1029B00074041CC01CC885475CC8F2406244D24401
:1029C00042490561828074003000AA84A53FA24577
:1029D0002A892685012219E98317C40013F70720E5
:1029E00069FFF19B93E727005EA4D1B7970700002A
:1029F0009387C7D99CD45E2408C008C893E707080A
:102A00005EA4A2475CC8B24781CF8315E400268547
:102A1000EF00501811C55E24F19B93E717005EA4E8
:102A20005E243369F9002316240141BFDDC183A769
:102A3000C5FF411122C406C626C21384C5FF63D355
:102A400007003E94AA84EF00B01B938781829C43C9
:102A500081EF2322040023A481822244B2402685F0
:102A6000924441016F00F019637EF4001440330773
:102A7000D4006396E7009843DC43369718C05CC0E7
:102A8000D9BFBA87D84319C3E37DE4FE94433386A4
:102A9000D700631F86001040B29694C33386D700D8
:102AA000E31DC7FA10435843B29694C3D8C375B711
:102AB0006375C400B1479CC04DB71040B306C40055
:102AC0006316D70014435843B29614C058C0C0C30D
:102AD00069B78280011126CA93843500F19806CE29
:102AE00022CC4AC84EC6A104B14763F3F404B144F2
:102AF00063E2B4042A89EF00B0109387818298437F
:102B00003A8439E09387C1829C4391E781454A85A5
:102B1000052F23A6A182A6854A851D27FD59631985
:102B20003507B1472320F9004A85EF00900D29A011
:102B3000E3D004FCB1471CC10145F2406244D244D9
:102B40004249B249056182801C40858F63CF0702EC
:102B5000AD4663F6F6001CC03E9404C031A05C4054
:102B60006313870223A4F1824A85EF0090091305BD
:102B7000B4009307440061993307F5405DDF3A9450
:102B8000898F1CC05DBF5CC3C5B72287404095BF1D
:102B9000130435007198E30285FCB305A4404A850F
:102BA0004525E31C35FBB5BF1C46FD171CC663DA83
:102BB0000700184E63C5E700A9476394F5006FF05E
:102BC0009F811C422E851387170018C28CA3828018
:102BD000011122CC26CA4AC84EC652C406CE2A8942
:102BE000AE893284B304D6007D5A63149400014543
:102BF00001A80C204E864A85453F0504E31745FF92
:102C0000F2406244D2444249B249224A056182807C
:102C1000357122CD26CB4AC94EC706CF52C556C301
:102C20005AC1DEDEE2DCE6DAAA89AE843289368475
:102C300001C51C4D91E34D36971700009387078916
:102C40006397F40C83A44900DE24A18BFDC39C4848
:102C5000EDC393070002A304F1029307000302D21D
:102C60002305F10222C6930B5002971A0000938AA3
:102C7000EA89054C294B4A841C2099C3639E770D31
:102C8000B30C2441638D0C00E6864A86A6854E85EA
:102C90008137FD57630FF51C9256E69636D21C20FD
:102CA0006389071CFD571309140002C802CE3ECAEF
:102CB00002CCA309010482D4834509001546568538
:102CC000252713041900C24751E913F7070109C763
:102CD00013070002A309E10413F7870009C71307CC
:102CE000B002A309E104834609001307A002638F21
:102CF000E606F2474A8481462546182093051400CB
:102D0000130707FD6377E60AB5CA3ECE85A8970785
:102D100000009387A77D6395F40083A489002DB7F5
:102D20009707000093878778E390F4F283A4C900A3
:102D300021BFA6854E85EFF0CFF501DD7D55FA4028
:102D40006A44DA444A49BA492A4A9A4A0A4BF65B23
:102D5000665CD65C0D618280050439BF3305554140
:102D60003315AC00C98F3EC82289B9B732479306E4
:102D70004700184336C6634707023ACE1820930728
:102D8000E002631DF70418309307A002631BF702EB
:102D9000B2470904138747009C433AC663C1070240
:102DA0003ECA2DA83307E04093E727003ACE3EC83D
:102DB000F1B7B387670385462E84BA973DBFFD57A9
:102DC000C5B7050402CA81468147254618209305E8
:102DD0001400130707FD6374E606F9F20C200D4694
:102DE0001705000013050573012511CD9707000095
:102DF000938747721D8D93070004B397A700424540
:102E000005045D8D2AC80C2019461705000013051E
:102E1000A570130914002304B102F92335C197D713
:102E2000FFFF9387271E95E74247B24713770710A6
:102E300009CF91073EC69257D2973ED22DBDB38798
:102E4000670385462E84BA9751B79D07E19BA1077A
:102E5000D5B77800970600009386C6D726860C085B
:102E60004E8597000000E7000000FD572A8AE31412
:102E7000F5FCDE2493F70704E39207EC1255C1B585
:102E80007800970600009386E6D426860C084E85C7
:102E9000012AE1BF797156CA9C49BA8A984522D461
:102EA00026D24ECE52CC06D64AD05AC85EC6AA8981
:102EB0002E84B284368A63D3E700BA879CC0034766
:102EC000340419C385079CC01C4093F7070281C7CF
:102ED0009C4089079CC00329040013796900631A88
:102EE0000900130B9401FD5B5C449840998F634C7F
:102EF000F9041C408346340493F70702B336D0002C
:102F0000A5EB13063404D2854E85829AFD576303E0
:102F1000F5041C4011469840998B544481446397B2
:102F2000C700B384E64063D3040081441C441848BE
:102F30006354F700998FBE94014969047D5B6398DF
:102F40002405014509A885465A86D2854E85829A70
:102F5000631E75017D55B250225492540259F249B4
:102F6000624AD24A424BB24B456182800509ADBFED
:102F70003307D40013060003A301C7040347540416
:102F800093871600A2978906A381E7049DBF854613
:102F90002286D2854E85829AE30E65FB050945B7E8
:102FA000797122D426D24AD04ECE06D652CC56CAF9
:102FB0005AC8B689942D930790063289AA842E8424
:102FC00013863504638DF60263E2D7069307800506
:102FD0006385F61863EDD700638D062093073004F0
:102FE000638EF60A930A24042301D404C9A093072C
:102FF00030066385F60A93074006E395F6FE1C400B
:10300000084393F6070893054500C5C61C410CC349
:1030100063D807001307D002B307F040A301E4040C
:10302000970600009386C64F294765A893070007B7
:103030006381F61663E5D7029307E0066388F61806
:103040009307F006E390F6FA0C401C4313F80508CA
:10305000138547006307080608C39C4385A89307A8
:103060005007E383F6FE930780076388F612930701
:103070003007E399F6F61C43D0418145938647001B
:1030800014C383AA07005685852601C5330555411B
:1030900048C05C401CC8A301040461A81C43930AF7
:1030A0002404938647009C4314C32301F4048547FA
:1030B000D5B793F607041C410CC3B9DAC207C18720
:1030C00081BF93F5050408C3C9D99E231307F006F1
:1030D0006386E60E97060000938686442947A3017F
:1030E00004044C400CC463C5050008406D9908C039
:1030F00099E3B28A89CDB28AB3F5E702FD1AB69593
:103100008C212380BA00B3D5E70263FFE70AA14709
:10311000631EF7001C40858B91CB58401C4863C749
:10312000E70093070003A38FFAFEFD1A330656410A
:1031300010C84E87CA867000A2852685A13B7D5A9D
:10314000631D450B7D55B250225492540259F249E9
:10315000624AD24A424B45618280A382D5049706D7
:1031600000009386E63B0C40084313F805081C4119
:103170001105630D080208C313F7150001C793E595
:1031800005020CC04147A1FF0C4093F5F5FD0CC0B2
:10319000B9B79C4193E707029CC193078007A3023C
:1031A000F404970600009386E63875BF13F805040B
:1031B00008C3E30308FCC207C1837DBF9706000074
:1031C00093860636214721BFAE873DB794411C4305
:1031D000CC4913F80608138547006306080008C3A6
:1031E0009C438CC339A008C393F606049C43F5DACC
:1031F0008EA323280400B28A2DBF14485686CA85A0
:1032000026858299E30045F51C40898B8DE7B247FE
:103210004844E35AF5F23E853DB785465686CA8551
:1032200026858299E30065F3050A5C443247998F4D
:10323000E345FAFEE9BF014A930A94017D5BF5B7C5
:10324000411122C42A842E8523AC018606C6EFE0F4
:10325000DF91FD576317F500938781879C4391C3E6
:103260001CC0B240224441018280411122C42E84FC
:103270008395E50006C67922634905007C48AA9734
:103280007CC8B2402244410182805E247D777D1754
:10329000F98F5EA4FDB7DE25011122CC26CA4AC8EB
:1032A0004EC606CE93F70710AA842E843289B689BB
:1032B00091C78395E5008946014609225E247D7702
:1032C0007D17F98F5EA48315E4006244F240CE8638
:1032D0004A86B24942492685D244056125A8411152
:1032E00022C42E848395E50006C6C928FD575A24BA
:1032F000631AF500FD77FD17F98F5EA4B2402244F2
:10330000410182808567D98F5EA468C8C5BF839557
:10331000E50005A8411122C42A842E85B28536868F
:1033200023AC018606C6EFE02FFDFD576317F500BD
:10333000938781879C4391C31CC0B24022444101C2
:103340008280411122C42A842E8523AC018606C6C0
:10335000C520FD576317F500938781879C4391C370
:103360001CC0B240224441018280411122C42A84FF
:103370002E85B28523AC018606C6C920FD5763178A
:10338000F500938781879C4391C31CC0B2402244BF
:1033900041018280411122C42A842E8523AC0186FA
:1033A00006C65D20FD576317F500938781879C4310
:1033B00091C31CC0B240224441018280411122C409
:1033C0002A842E85B285368623AC018606C659200E
:1033D000FD576317F500938781879C4391C31CC0F9
:1033E000B24022444101828093F5F50F2A9663147E
:1033F000C500014582801C21E38EB7FE0505C5BFCF
:1034000082808280411122C42A842E85B28536862C
:1034100023AC018606C6A920FD576317F5009387E4
:1034200081879C4391C31CC0B240224441018280E9
:103430009307800523ACF1867D5582809307800534
:1034400023ACF1867D5582809307800523ACF186FD
:10345000014582809307800523ACF1867D558280EB
:103460009307800523ACF1867D5582805379737470
:10347000656D436C6B3A2564090A000054686973F2
:10348000206973207072696E7466206578616D7052
:103490006C650D0072656400677265656E00000002
:1034A000626C756500000000000000000000000074
:1034B000000000000000000000000000000000000C
:1034C00000000000000000000000000000000000FC
:1034D00000000000000000000000000000000000EC
:1034E00000000000000000000000000000000000DC
:1034F00000000000000000000000000000000000CC
:103500000000000000000000232D302B20000000F0
:10351000686C4C00656667454647000030313233C1
:1035200034353637383941424344454600000000BF
:103530003031323334353637383961626364656629
:043540000000000087
:103544000000000001020304010203040607080945
:1035540000000000C8340000E8340000A834000073
:103564000000000000000000000000000000000057
:103574000000000000000000000000000000000047
:103584000000000000000000000000000000000037
:103594000000000000000000000000000000000027
:1035A4000000000000000000000000000000000017
:1035B40000D8B80502040608EC0000201000002022
:0835C4001000002000000000CF
:00000001FF
